:020000040800F2
:1000000000200020152700082527000825270008C4
:1000100000000000000000000000000000000000E0
:10002000000000000000000000000000252700087C
:100030000000000000000000252700082527000818
:100040002527000825270008252700082527000860
:100050002527000825270008252700082527000850
:100060002527000825270008252700082527000840
:100070002527000825270008252700082527000830
:100080002527000825270008000000002527000874
:100090002527000825270008252700082527000810
:1000A0002527000825270008252700082527000800
:1000B0002527000800000000252700080000000098
:0400C0005FF808F1EC
:1000C80080B500AF1B4B1B4A126801210A431A6016
:1000D800184B184A526818490A405A60154B154A75
:1000E800126816490A401A60124B124A12681449DB
:1000F8000A401A600F4B0F4A526812490A405A6068
:100108000C4B0C4AD26A0F218A43DA62094B094A1E
:10011800126B0D490A401A63064B064A526B0121BD
:100128008A435A63034B00229A6000F079F8BD466F
:1001380080BDC046001002400CB8FF08FFFFF6FE65
:10014800FFFFFBFFFFFFC0FFACFEFFFF80B584B0E1
:1001580000AF0023FB600023BB6000237B6000230B
:100168003B602A4B5B680C221340FB60FB68042B46
:1001780007D0082B09D0002B31D1254B254A1A600E
:1001880031E0234B234A1A602DE0204B5A68F023B4
:100198009B031340BB601D4B5A68C0235B0213408E
:1001A8007B60BB689B0C0233BB607B68002B05D16E
:1001B800BB68194A5A43164B1A6014E0134BDB6AA2
:1001C8000F22134001333B601248396802F0A8FA45
:1001D800031C1A1CBB685A430D4B1A6003E00C4BF6
:1001E8000C4A1A60C046094B5B68F02213401B0991
:1001F8000A4AD35CDBB2FB60054B1A68FB68DA403D
:10020800034B1A60BD4604B080BDC04600100240D2
:100218000000002000127A0000093D0004000020C0
:1002280080B582B000AF00237B6000233B60314B78
:10023800304A1268802149020A431A602D4B1A6815
:1002480080239B0213403B607B6801337B603B68E3
:10025800002B04D17A68A023DB019A42EED1254B0A
:100268001A6880239B02134002D001233B6001E0FF
:1002780000233B603B68012B38D11F4B11221A60C9
:100288001C4B1C4A52685A601A4B1A4A52685A60E8
:10029800184B184A526819490A405A60154B154AB2
:1002A8005268882149030A435A60124B114A12685E
:1002B800802149040A431A60C0460E4B1A688023FD
:1002C8009B041340F9D00B4B0A4A526803218A4316
:1002D8005A60084B074A526802210A435A60C046CE
:1002E800044B5B680C221340082BF9D1BD4602B0C1
:1002F80080BDC0460010024000200240FF7FC0FFC2
:1003080080B500AF1A4B1A4A126801210A431A60D5
:10031800174B174A526817490A405A60144B144A37
:10032800126815490A401A60114B114A126813499C
:100338000A401A600E4B0E4A526811490A405A6028
:100348000B4B0B4AD26A0F218A43DA62084B084AE0
:10035800126B0C490A401A63054B054A526B01217E
:100368008A435A63024B00229A60BD4680BDC0464C
:10037800001002400CB8FF08FFFFF6FEFFFFFBFF6E
:10038800FFFFC0FFACFEF0FF80B582B000AF021CDB
:10039800FB1D1A70044B00221A70034AFB1D1B78C0
:1003A8001370BD4602B080BD0210024090B583B004
:1003B80000AF00233B60FB1D00221A70BB1D00220A
:1003C8001A70BC1D112000F03FFD031C23703B6810
:1003D80001333B603A68A023DB019A4203D0BB1D7E
:1003E8001B78002BEDD0112000F02EFD031E03D04A
:1003F800FB1D01221A7002E0FB1D00221A70FB1D72
:100408001B78181CBD4603B090BDC04680B584B0AB
:1004180000AF021CFB1D1A700023FB60094B1B6810
:10042800FB60FB68F8229343FB60FB1D1B78DB0035
:10043800FA681343FB60034BFA681A60BD4604B0C0
:1004480080BDC0460010024080B582B000AF021CDB
:10045800FB1D1A70FB1D1B78002B06D0074B074AA3
:10046800126801210A431A6005E0044B034A126826
:1004780001218A431A60BD4602B080BD00100240C7
:1004880080B584B000AF021CFB1D1A700023FB600E
:10049800094B5B6BFB60FB68F8229343FB60FB1D19
:1004A8001B78DB00FA681343FB60034BFA685A6356
:1004B800BD4604B080BDC0460010024080B582B081
:1004C80000AF021CFB1D1A70FB1D1B78002B06D009
:1004D800074B074A526B01210A435A6305E0044B54
:1004E800034A526B01218A435A63BD4602B080BD5C
:1004F8000010024080B582B000AF021CFB1D1A70CC
:10050800FB1D1B78002B06D0074B074A526B0421B2
:100518008A435A6305E0044B034A526B04210A4399
:100528005A63BD4602B080BD0010024080B582B05B
:1005380000AF78600A4B0A4A126A01218A431A629C
:10054800074B074A126A04218A431A62044B044A79
:10055800116A7A680A431A62BD4602B080BDC04675
:100568000010024080B582B000AF7860074B074AA0
:10057800126A18218A431A62044B044A116A7A687B
:100588000A431A62BD4602B080BDC0460010024050
:1005980080B582B000AF021CFB1D1A70FB1D1B78D2
:1005A800002B06D0074B074A526A01210A435A62B8
:1005B80005E0044B034A526A01218A435A62BD4648
:1005C80002B080BD0010024080B582B000AF7860F4
:1005D8003960084B074A526807490A405A60054B78
:1005E800044A516878683A6802430A435A60BD462B
:1005F80002B080BD00100240FF7FC2FF80B582B00C
:1006080000AF021CFB1D1A70FB1D1B78002B07D0C6
:10061800084B084A1268802149040A431A6005E019
:10062800044B044A126804490A401A60BD4602B0E5
:1006380080BDC04600100240FFFFFFFE80B582B0BB
:1006480000AF021CFB1D1A70FB1D1B78002B07D086
:10065800084B084A526B802149020A435A6305E055
:10066800044B044A526B04490A405A63BD4602B01F
:1006780080BDC04600100240FFFFFEFF80B584B079
:1006880000AF78600023FB60084BDB6AFB60FB6807
:100698000F229343FB60FA687B681343FB60034BAC
:1006A800FA68DA62BD4604B080BDC0460010024058
:1006B80080B582B000AF021CFB1D1A70FB1D1B78B1
:1006C800002B07D0084B084A1268802109030A4307
:1006D8001A6005E0044B044A126804490A401A608B
:1006E800BD4602B080BDC04600100240FFFFF7FFC4
:1006F80080B584B000AF021C3960FB1D1A7000235E
:10070800FB600A4B5B68FB60FB681B021B0AFB6013
:10071800FB1D1B781A063B681343FA681343FB60FA
:10072800024BFA685A60BD4604B080BD0010024012
:1007380080B584B000AF78600023FB60084B5B682D
:10074800FB60FB6803229343FB60FA687B681343F2
:10075800FB60034BFA685A60BD4604B080BDC046D2
:100768000010024080B500AF044B5B68DBB20C227E
:100778001340DBB2181CBD4680BDC04600100240C5
:1007880080B584B000AF78600023FB60084B5B68DD
:10079800FB60FB68F0229343FB60FA687B681343B5
:1007A800FB60034BFA685A60BD4604B080BDC04682
:1007B8000010024080B584B000AF78600023FB6071
:1007C800084B5B68FB60FB68074A1340FB60FA68EC
:1007D8007B681343FB60034BFA685A60BD4604B05C
:1007E80080BDC04600100240FFF8FFFF80B582B010
:1007F80000AF78600E4B0E4A52680E490A405A60A4
:100808000B4B0B4A51687A681204120C0A435A605F
:10081800074B074A126B08490A401A63044B044AFB
:10082800116B7A68120C0A431A63BD4602B080BD88
:1008380000100240FFBFFFFFFFFEFFFF80B582B040
:1008480000AF7860074B074A126B40218A431A634E
:10085800044B044A116B7A680A431A63BD4602B016
:1008680080BDC0460010024080B582B000AF7860FD
:10087800074B074A126B10218A431A63044B044A38
:10088800116B7A680A431A63BD4602B080BDC04640
:100898000010024080B584B000AF78600023FB6090
:1008A8007B681B0FFB60FB68012B06D10F4B0F4ABF
:1008B800126B03218A431A630FE0FB68022B06D1EF
:1008C8000A4B0A4A126B0A490A401A6305E0074BA9
:1008D800064A126B07490A401A63044B034A116B14
:1008E8007A680A431A63BD4604B080BD001002400E
:1008F800FFFFFCFFFFFFF3FF80B582B000AF786019
:10090800074B074A126B80218A431A63044B044A37
:10091800116B7A680A431A63BD4602B080BDC046AF
:100928000010024080B588B000AF78600023BB613A
:1009380000237B6100233B610023FB600023BB6035
:100948000023FB61A34B5B680C221340BB61BB69AE
:10095800042B0CD002D8002B05D03BE0082B0AD082
:100968000C2B33D036E07B689B4A1A6036E07B68F4
:10097800994A1A6032E0974B5A68F0239B03134058
:100988007B61944B5A68C0235B0213403B617B69CF
:100998009B0C02337B613B69002B04D17B698F4A36
:1009A8005343FB610EE08B4BDB6A0F22134001338C
:1009B800FB608948F96801F0B3FE031C1A1C7B69C7
:1009C8005343FB617B68FA691A6007E07B68844AD5
:1009D8001A6003E07B68804A1A60C0467D4B5B68FA
:1009E800F0221340BB61BB691B09BB617D4ABB692F
:1009F800D3181B78DBB2BB607B681A68BB68DA4027
:100A08007B685A60734B5A68E023DB001340BB6174
:100A1800BB691B0ABB61734ABB69D3181B78DBB27D
:100A2800BB607B685A68BB68DA407B689A60694B30
:100A38001A6B80235B00134003D17B686A4ADA6033
:100A480010E0644B5A688023DB01134005D17B68B2
:100A58009B685A087B68DA6004E07B689B689A08A0
:100A68007B68DA605B4B1B6B4022134003D17B68C9
:100A78005E4A1A6103E07B68802212021A61554BB4
:100A88001B6B1022134003D17B68534A5A6103E061
:100A98007B681A687B685A614E4B1B6B03221340B4
:100AA80004D17B689A687B689A611EE0494B1B6B8E
:100AB80003221340012B04D17B681A687B689A6172
:100AC80013E0444B1B6B03221340022B04D17B68B9
:100AD800802212029A6108E03E4B1B6B03221340EE
:100AE800032B02D17B683C4A9A613A4B1A6BC023AC
:100AF8009B02134004D17B689A687B68DA6127E01F
:100B0800344B1A6BC0239B021A4080235B029A4223
:100B180004D17B681A687B68DA6119E02D4B1A6B7F
:100B2800C0239B021A4080239B029A4204D17B680F
:100B380080221202DA610BE0264B1A6BC0239B025B
:100B48001A40C0239B029A4202D17B68224ADA618A
:100B5800204B1A6BC0231B03134004D17B689A688F
:100B68007B681A6227E01B4B1A6BC0231B031A40D1
:100B78008023DB029A4204D17B681A687B681A6278
:100B880019E0144B1A6BC0231B031A4080231B0364
:100B98009A4204D17B68802212021A620BE00D4B44
:100BA8001A6BC0231B031A40C0231B039A4202D1AD
:100BB8007B68094A1A62074B1B6B8022134003D1DA
:100BC8007B68074A5A6202E07B68FA695A62BD4646
:100BD80008B080BD0010024000127A0000093D00F4
:100BE800006CDC0214000020809FD50012800000F9
:100BF80080B582B000AF7860044B044A116A7A6805
:100C08000A431A62BD4602B080BDC04600100240C9
:100C180080B582B000AF021CFB1D1A70FB1D1B784B
:100C2800002B07D0084B084A126A802109020A43A0
:100C38001A6205E0044B044A126A04490A401A621F
:100C4800BD4602B080BDC04600100240FF7FFFFFD6
:100C580080B582B000AF021CFB1D1A70FB1D1B780B
:100C6800002B07D0084B084A126A802149020A4320
:100C78001A6205E0044B044A126A04490A401A62DF
:100C8800BD4602B080BDC04600100240FFFFFEFF17
:100C980080B582B000AF78600A1CFB1C1A70FB1C80
:100CA8001B78002B06D0084B074A51697A680A431B
:100CB8005A6106E0044B044A52697968C9430A40FC
:100CC8005A61BD4602B080BD0010024080B582B0B6
:100CD80000AF78600A1CFB1C1A70FB1C1B78002BE9
:100CE80006D0084B074A91697A680A439A6106E078
:100CF800044B044A92697968C9430A409A61BD461F
:100D080002B080BD0010024080B582B000AF7860AC
:100D18000A1CFB1C1A70FB1C1B78002B06D0084B06
:100D2800074AD1697A680A43DA6106E0044B044A43
:100D3800D2697968C9430A40DA61BD4602B080BD0C
:100D48000010024080B582B000AF78600A1CFB1C1E
:100D58001A70FB1C1B78002B06D0084B074A916AB7
:100D68007A680A439A6206E0044B044A926A7968F0
:100D7800C9430A409A62BD4602B080BD00100240D5
:100D880080B582B000AF78600A1CFB1C1A70FB1C8F
:100D98001B78002B06D0084B074AD1687A680A43AB
:100DA800DA6006E0044B044AD2687968C9430A400D
:100DB800DA60BD4602B080BD0010024080B582B046
:100DC80000AF78600A1CFB1C1A70FB1C1B78002BF8
:100DD80006D0084B074A11697A680A431A6106E087
:100DE800044B044A12697968C9430A401A61BD462E
:100DF80002B080BD0010024080B582B000AF021C76
:100E0800FB1D1A70BB1D0A1C1A70BB1D1B78002B1A
:100E180009D00C490B4B1B78DAB2FB1D1B78134326
:100E2800DBB20B700AE00749064B1B78DBB2FA1DF0
:100E38001278D243D2B21340DBB20B70BD4602B077
:100E480080BDC0460910024080B586B000AF021CC4
:100E5800FB1D1A700023FB6000237B611323FB1822
:100E680000221A70FB1D1B785B09DBB2FB60FB6874
:100E7800002B03D1184B1B687B6110E0FB68012B2A
:100E880003D1154B1B6A7B6109E0FB68022B03D178
:100E9800114B5B6A7B6102E00F4B5B6B7B61FB1D57
:100EA8001B781F221340FB60FB687A69DA40131C29
:100EB8000122134004D01323FB1801221A7003E007
:100EC8001323FB1800221A701323FB181B78181C15
:100ED800BD4606B080BDC0460010024080B500AFD8
:100EE800044B044A526A802149040A435A62BD46A7
:100EF80080BDC0460010024080B584B000AF021C1F
:100F0800FB1D1A700F23FB1800221A700A4B9B68EE
:100F1800FA1D1278134004D00F23FB1801221A700F
:100F280003E00F23FB1800221A700F23FB181B780D
:100F3800181CBD4604B080BD0010024080B582B0C8
:100F480000AF021CFB1D1A70034AFB1D1B781370AF
:100F5800BD4602B080BDC0460A10024080B582B0CE
:100F680000AF78607A689023DB059A420CD1802321
:100F78009B02181C0121FFF7E5FE80239B02181C29
:100F88000021FFF7DFFE53E07B682B4A93420CD128
:100F98008023DB02181C0121FFF7D4FE8023DB022B
:100FA800181C0021FFF7CEFE42E07B68234A9342DB
:100FB8000CD180231B03181C0121FFF7C3FE8023DB
:100FC8001B03181C0021FFF7BDFE31E07B681C4A9B
:100FD80093420CD180235B03181C0121FFF7B2FE5A
:100FE80080235B03181C0021FFF7ACFE20E07B6820
:100FF800144A93420CD180239B03181C0121FFF74C
:10100800A1FE80239B03181C0021FFF79BFE0FE025
:101018007B680D4A93420BD18023DB03181C012106
:10102800FFF790FE8023DB03181C0021FFF78AFEE0
:10103800BD4602B080BDC046000400480008004814
:10104800000C0048001000480014004880B586B025
:1010580000AF7860396000237B6100233B61002387
:10106800FB6000237B617CE07B6901229A40131CB2
:101078003B613B681B683A691340FB60FA683B694F
:101088009A426BD13B681B79012B03D03B681B79D3
:10109800022B34D17B689B687A695200111C0322A9
:1010A8008A40D2431A407B689A607B689A683B689A
:1010B8005B79191C7B695B0099400B1C1A437B68A0
:1010C8009A607B689B889BB27A6992B2111C012254
:1010D8008A4092B2D24392B213409AB27B689A8005
:1010E8007B689B889AB23B689B79191C7B699BB289
:1010F80099400B1C9BB213439AB27B689A807B6819
:101108001B687A695200111C03228A40D2431A4094
:101118007B681A607B681A683B681B79191C7B69B5
:101128005B0099400B1C1A437B681A607B68DB687C
:101138007A6992B25200032191400A1CD2431A40A4
:101148007B68DA607B68DA683B68DB79191C7B6945
:101158005B0099400B1C1A437B68DA607B6901339A
:101168007B617B690F2B00D87EE7BD4606B080BD4A
:1011780080B582B000AF78607B68084A1A607B68E7
:1011880000221A717B6801225A717B6800229A71C9
:101198007B680022DA71BD4602B080BDFFFF000007
:1011A80080B584B000AF78600A1CBB1C1A8080230D
:1011B8005B02FB60BB1C1A88FB681343FB60FA6880
:1011C8007B68DA61BB1C1A887B68DA61FA687B681D
:1011D800DA617B68DB69FB607B68DB69FB60BD46C5
:1011E80004B080BD80B584B000AF78600A1CBB1C19
:1011F8001A800F23FB1800221A707B681B8A9BB287
:10120800BA1C128813409BB2002B04D00F23FB1882
:1012180001221A7003E00F23FB1800221A700F2313
:10122800FB181B78181CBD4604B080BD80B582B081
:1012380000AF78607B681B8A9BB2181CBD4602B061
:1012480080BDC04680B584B000AF78600A1CBB1C66
:101258001A800F23FB1800221A707B689B8A9BB2A6
:10126800BA1C128813409BB2002B04D00F23FB1822
:1012780001221A7003E00F23FB1800221A700F23B3
:10128800FB181B78181CBD4604B080BD80B582B021
:1012980000AF78607B689B8A9BB2181CBD4602B081
:1012A80080BDC04680B582B000AF78600A1CBB1C08
:1012B8001A80BB1C1A887B689A61BD4602B080BD43
:1012C80080B582B000AF78600A1CBB1C1A807B68AE
:1012D800BA1C12881A85BD4602B080BD80B582B09E
:1012E80000AF7860081C111CBB1C021C1A807B1CF8
:1012F8000A1C1A707B1C1B78002B04D0BB1C1A8894
:101308007B689A6103E07B68BA1C12881A85BD461F
:1013180002B080BD80B582B000AF78600A1CBB1CEB
:101328001A807B68BA1C12889A82BD4602B080BDBA
:1013380080B584B000AF7860081C111CBB1C021C6F
:101348001A807B1C0A1C1A700023FB600023BB60F8
:101358007B1C1B78BA1C128807210A409200934014
:10136800FB60BB1C1B88DB089BB2181CBB1C1B88C2
:10137800DB089BB21A1C7B6808329200D358BA1C4F
:10138800128807210A409200111C0F228A40D2437A
:101398001A40111C7B68021C08329200D150BB1CF9
:1013A8001B88DB089BB21A1C7B6808329200D25853
:1013B800FB681343BB60BB1C1B88DB089BB21A1C71
:1013C8007B6808329200B968D150BD4604B080BD30
:1013D80080B582B000AF78607B68114A93420CD127
:1013E80080235B01181C0121FFF7CAFC80235B01E5
:1013F800181C0021FFF7C4FC0FE07B68094A9342E0
:101408000BD18023DB01181C0121FFF7D7FC8023B7
:10141800DB01181C0021FFF7D1FCBD4602B080BDDE
:10142800003001400038004080B582B000AF7860DD
:101438007B6800221A807B6800225A807B68E02241
:10144800D2009A807B680022DA807B6800221A81A9
:101458007B6800225A817B6800229A817B6800227F
:10146800DA817B6807221A82BD4602B080BDC04679
:1014780080B584B000AF786039600E23FB18002275
:101488001A800E23FB187A6812881A800E23FB181C
:101498000E22BA181188C12292010A401A803B68AC
:1014A8001A883B68DB8913439AB23B68DB8813438D
:1014B8009AB23B681B8913439AB23B685B89134312
:1014C8009AB23B689B89134399B20E23FB180E22EC
:1014D800BA1812880A431A807B680E22BA18128832
:1014E8001A800E23FB187A6892881A800E23FB183C
:1014F8000E22BA1812881D490A401A803B6899883A
:101508000E23FB180E22BA1812880A431A807B6829
:101518000E22BA1812889A803B681A8A7B681A8247
:101528000E23FB187A6812881A800E23FB180E22E5
:10153800BA18128804218A431A803B6859880E23F6
:10154800FB180E22BA1812880A431A807B680E22EA
:10155800BA1812881A807B689B8B9BB2044A134086
:101568009AB27B689A83BD4604B080BDFFF0FFFF46
:10157800FFF7FFFF80B582B000AF78607B6800227C
:101588001A807B6800225A807B6800229A807B68D8
:101598000022DA807B6802229A607B6800229A81A6
:1015A800BD4602B080BDC04680B592B000AF78603D
:1015B80039603A23FB1800221A804623FB180222BE
:1015C8001A804423FB1800221A804223FB180122A8
:1015D8001A800023FB6300237B637B689B8B9BB291
:1015E800604A13409AB27B689A837B6802221A8405
:1015F8003A23FB187A68928B1A803B689B68022B07
:1016080008D14423FB1800221A804623FB18022223
:101618001A8066E03B689B88002B04D14223FB18A4
:1016280001221A8003E04223FB1802221A800C23AD
:10163800FB18181CFFF776F90C23FB181B687B6353
:101648003B68DA8880239B009A4212D17B6B1A0A86
:10165800131C9B009B185B001A1C3B689B68101CA2
:10166800191C01F05DF8031C9BB205339BB2FB63A8
:1016780019E04223FB181B885B01786B191C01F0E9
:101688004FF8031C1A1C131C9B009B185B001A1CA8
:101698003B689B68101C191C01F042F8031C9BB2A4
:1016A80005339BB2FB63FB6B181C0A2101F038F869
:1016B800031CFB63FB6B9AB24423FB1801210A400D
:1016C8001A804423FB181B88FA6BD31A5A0846233E
:1016D800FB181A804423FB184422BA1812881202F5
:1016E8001A804623FB181B88012B04D94623FB18B4
:1016F8001B88FF2B07D94623FB1802221A80442394
:10170800FB1800221A803B68DA884423FB181B88E0
:1017180013439AB24623FB181B8813439AB27B687B
:101728001A843B681A883B6859883B6898883B68E4
:101738009B8903439BB20B439BB213439AB23A2350
:10174800FB181B8813439AB23A23FB18802109011E
:101758000A431A807B683A22BA1812889A83BD46CF
:1017680012B080BD40F0FFFF80B582B000AF786056
:101778000A1CFB1C1A70FB1C1B78002B08D07B680A
:101788001B889BB2402213439AB27B681A8007E0F9
:101798007B681B889BB2402293439AB27B681A806D
:1017A800BD4602B080BDC04680B582B000AF78604B
:1017B8000A1CFB1C1A70FB1C1B78002B08D07B68CA
:1017C8009B889BB2102213439AB27B689A8007E0E9
:1017D8007B689B889BB2102293439AB27B689A805D
:1017E800BD4602B080BDC04680B582B000AF78600B
:1017F8000A1CFB1C1A70FB1C1B78002B09D07B6889
:101808009B8B9BB28022D20013439AB27B689A8347
:1018180007E07B689B8B9BB2034A13409AB27B68B4
:101828009A83BD4602B080BDFFFBFFFF80B584B040
:1018380000AF78600A1CBB1C1A800E23FB1800221C
:101848001A800E23FB187A6892881A800E23FB18D8
:101858000E22BA1812880A490A401A800E23FB1869
:101868000E22B918BA1C098812880A431A807B68A4
:101878000E22BA1812889A80BD4604B080BDC046B0
:10188800FFF0FFFF80B582B000AF78600A1CBB1C78
:101898001A807B689B889BB2084A13409AB27B687F
:1018A8009A807B689B889AB2BB1C1B8813439AB2A8
:1018B8007B689A80BD4602B080BDC046FFEFFFFF3F
:1018C80080B582B000AF78600A1CBB1C1A80BB1CB4
:1018D8001A888023DB019A4209D17B681B889BB256
:1018E8008022D20113439AB27B681A8007E07B6892
:1018F8001B889BB2034A13409AB27B681A80BD4684
:1019080002B080BDFFBFFFFF80B582B000AF786036
:101918000A1CBB1C1A80BB1C1B880C4A934209D0AA
:101928007B681B889BB28022520013439AB27B6863
:101938001A8007E07B681B889BB2054A13409AB25D
:101948007B681A80BD4602B080BDC046FFFE00001D
:10195800FFFEFFFF80B582B000AF78600A1CFB1C59
:101968001A70FB1C1B78002B08D07B689B889BB2E5
:10197800042213439AB27B689A8007E07B689B88AD
:101988009BB2042293439AB27B689A80BD4602B008
:1019980080BDC04680B582B000AF78600A1CFB1CD1
:1019A8001A70FB1C1B78002B08D07B689B889BB2A5
:1019B800082213439AB27B689A8007E07B689B8869
:1019C8009BB2082293439AB27B689A80BD4602B0C4
:1019D80080BDC04680B584B000AF78600A1CFB1C8F
:1019E8001A700023FB607B68FB60FB680C33FB60AC
:1019F800FB68FA1C12781A70BD4604B080BDC04658
:101A080080B582B000AF78600A1CBB1C1A807B6866
:101A1800BA1C12889A81BD4602B080BD80B584B0D8
:101A280000AF78600023FB607B68FB60FB680C33C9
:101A3800FB60FB681B78DBB2181CBD4604B080BD98
:101A480080B582B000AF78607B689B899BB2181C18
:101A5800BD4602B080BDC04680B582B000AF786098
:101A68000A1CBB1C1A807B681B889BB2084A13405F
:101A78009AB27B681A807B681B889AB2BB1C1B8849
:101A880013439AB27B681A80BD4602B080BDC04637
:101A9800FFF7FFFF80B582B000AF78600A1CFB1C1F
:101AA8001A70FB1C1B78002B09D07B681B889BB223
:101AB8008022920113439AB27B681A8007E07B6800
:101AC8001B889BB2034A13409AB27B681A80BD46B2
:101AD80002B080BDFFDFFFFF80B582B000AF786045
:101AE8007B681B889BB28022520113439AB27B68A1
:101AF8001A80BD4602B080BD80B584B000AF786062
:101B08000A1CFB1C1A700E23FB1800221A80FB1CEF
:101B18001B78012B05D00E23FB187A68128B1A80CC
:101B280004E00E23FB187A68928A1A800E23FB18A9
:101B38001B88181CBD4604B080BDC04680B582B065
:101B480000AF78607B681B8A9BB2181CBD4602B048
:101B580080BDC04680B582B000AF7860081C111CFB
:101B6800BB1C021C1A807B1C0A1C1A707B1C1B786D
:101B7800002B09D07B689B889AB2BB1C1B88134337
:101B88009AB27B689A800AE07B689B889BB2BA1CF1
:101B98001288D24392B213409AB27B689A80BD46AB
:101BA80002B080BD80B582B000AF78600A1CBB1C53
:101BB8001A807B689B889BB2084A13409AB27B685C
:101BC8009A807B689B889AB2BB1C1B8813439AB285
:101BD8007B689A80BD4602B080BDC046FF9FFFFF6C
:101BE80080B584B000AF7860081C111CFB1C021C77
:101BF8001A70BB1C0A1C1A700E23FB1800221A80CC
:101C08000C23FB1800221A80FB1C1B781B09DAB274
:101C18000E23FB181A800E23FB181B8801229A40FA
:101C28000C23FB181A80BB1C1B78002B0AD07B687E
:101C38009B889AB20C23FB181B8813439AB27B68C3
:101C48009A800BE07B689B889BB20C22BA1812889A
:101C5800D24392B213409AB27B689A80BD4604B0D0
:101C680080BDC04680B582B000AF78607B681B89B4
:101C78009AB2C0235B0113409BB2181CBD4602B048
:101C880080BDC04680B582B000AF78607B681B8994
:101C98009AB2C023DB0013409BB2181CBD4602B0A9
:101CA80080BDC04680B584B000AF78600A1CBB1CFC
:101CB8001A800F23FB1800221A707B681B899BB2BD
:101CC800BA1C128813409BB2002B04D00F23FB18B8
:101CD80001221A7003E00F23FB1800221A700F2349
:101CE800FB181B78181CBD4604B080BD80B582B0B7
:101CF80000AF78600A1CBB1C1A80BB1C1B88DB4326
:101D08009AB27B681A81BD4602B080BD80B584B0A6
:101D180000AF78600A1CFB1C1A700F23FB18002206
:101D28001A700C23FB1800221A800A23FB180022C1
:101D38001A800823FB1800221A80FB1C1B780F222C
:101D4800134001229A400C23FB181A80FB1C1B78B5
:101D58001B09DAB20A23FB181A800A23FB181B880E
:101D680001229A400A23FB181A807B689B889AB242
:101D78000823FB180A21791809880A401A807B6809
:101D88001B899BB20C22BA18128813409BB2002BF5
:101D980009D00823FB181B88002B04D00F23FB183D
:101DA80001221A7003E00F23FB1800221A700F2378
:101DB800FB181B78181CBD4604B080BD80B582B0E6
:101DC80000AF78607B68094A93420BD180239B005F
:101DD800181C0121FEF7D4FF80239B00181C00214A
:101DE800FEF7CEFFBD4602B080BDC04600240140CC
:101DF80080B584B000AF786039600023FB607B68F1
:101E0800DB68FB60FB680F4A1340FB603B681A689D
:101E18003B681B795B031A433B689B681A433B6822
:101E2800DB681A433B681B691A433B685B691343C9
:101E3800FA681343FB607B68FA68DA60BD4604B051
:101E480080BDC04603D2FFFF80B582B000AF786086
:101E58007B6800221A607B6800221A717B68002266
:101E68009A607B680022DA607B6800221A617B68CE
:101E780000225A61BD4602B080BDC04680B582B01E
:101E880000AF78600A1CFB1C1A70FB1C1B78002B27
:101E980006D07B689B6801221A437B689A6005E03C
:101EA8007B689B6802221A437B689A60BD4602B031
:101EB80080BDC04680B582B000AF786039607B686D
:101EC8003A681A61BD4602B080BDC04680B584B08C
:101ED80000AFF860B960FB1D1A70FB1D1B78002B62
:101EE80006D0FB681A69BB681A43FB681A6106E0EA
:101EF800FB681B69BA68D2431A40FB681A61BD4681
:101F080004B080BD80B582B000AF78600A1CFB1CAD
:101F18001A70FB1C1B78002B07D07B68DB688022BB
:101F280012021A437B68DA6005E07B68DB68034AC3
:101F38001A407B68DA60BD4602B080BDFF7FFFFFB4
:101F480080B582B000AF78600A1CFB1C1A70FB1CBD
:101F58001B78002B07D07B68DB688022D2011A43EC
:101F68007B68DA6005E07B68DB68034A1A407B68B7
:101F7800DA60BD4602B080BDFFBFFFFF80B582B00A
:101F880000AF78600A1CFB1C1A70FB1C1B78002B26
:101F980007D07B68DB68802212041A437B68DA600A
:101FA80005E07B68DB68034A1A407B68DA60BD4657
:101FB80002B080BDFFFF7FFF80B582B000AF7860C0
:101FC800081C111CBB1C021C1A803B1C0A1C1A8012
:101FD8003B1C1A88BB1C1B881B041A437B681A62AB
:101FE800BD4602B080BDC04680B584B000AF786001
:101FF80039600023FB607B68DB68FB60FB68064A8E
:102008001340FB60FA683B681343FB607B68FA681F
:10201800DA60BD4604B080BDFFFFFF8380B582B0A3
:1020280000AF78600A1CFB1C1A70FB1C1B78002B85
:1020380007D07B68DB688022D2031A437B68DA60AA
:1020480005E07B68DB68034A1A407B68DA60BD46B6
:1020580002B080BDFFFFBFFF80B582B000AF021C99
:10206800FB1D1A70FB1D1B78002B07D0084B084A74
:102078001268802109040A431A6005E0044B044AE7
:10208800126804490A401A60BD4602B080BDC046C5
:1020980008270140FFFF7FFF80B582B000AF021C18
:1020A800FB1D1A70FB1D1B78002B07D0084B084A34
:1020B80012688021C9030A431A6005E0044B044AE8
:1020C800126804490A401A60BD4602B080BDC04685
:1020D80008270140FFFFBFFF80B582B000AF021C98
:1020E800FB1D1A70FB1D1B78002B07D0084B084AF4
:1020F8001268802149040A431A6005E0044B044A27
:10210800126804490A401A60BD4602B080BDC04644
:1021180008270140FFFFFFFE80B586B000AFF860DA
:10212800B9607A6000237B61FB689A6ABB681A43CE
:10213800FB689A627B69072293437B617A697B68B3
:1021480013437B61FB687A695A61BD4606B080BD5E
:1021580080B582B000AF78600A1CFB1C1A70FB1CAB
:102168001B78002B07D07B68DB68802292011A431A
:102178007B68DA6005E07B68DB68034A1A407B68A5
:10218800DA60BD4602B080BDFFDFFFFF80B582B0D8
:1021980000AF78600A1CFB1C1A70FB1C1B78002B14
:1021A80007D07B68DB68802252021A437B68DA60BA
:1021B80005E07B68DB68034A1A407B68DA60BD4645
:1021C80002B080BDFFFFFEFF80B582B000AF78602F
:1021D8000A1CFB1C1A70FB1C1B78002B07D07B68A1
:1021E800DB68802252011A437B68DA6005E07B686D
:1021F800DB68034A1A407B68DA60BD4602B080BDDE
:10220800FFEFFFFF80B586B000AF786000237B61E9
:1022180000233B610023FB607B689B6880221206D9
:102228001A437B689A607B689B68DB0FDB07FB605F
:102238003B6901333B613A69F0231B029A4202D0A1
:10224800FB68002BEFD17B689B68002B03DB7B6866
:102258001B6C7B6101E000237B617B69181CBD4618
:1022680006B080BD80B582B000AF78607B689B689F
:1022780010221A437B689A60BD4602B080BDC046F2
:1022880080B582B000AF78607B689B6804221A43EF
:102298007B689A60BD4602B080BDC04680B582B0FA
:1022A80000AF78607B681B6C9BB2181CBD4602B0FF
:1022B80080BDC04680B582B000AF78600A1CFB1CA8
:1022C8001A70FB1C1B78002B06D07B68DB68012288
:1022D8001A437B68DA6006E07B68DB680122934377
:1022E8001A1C7B68DA60BD4602B080BD80B582B03A
:1022F80000AF786039607B68DB68022293431A1C60
:102308007B68DA607B68DA683B681A437B68DA6066
:10231800BD4602B080BDC04680B584B000AFF8604D
:10232800B960FB1D1A70FB1D1B78002B06D0FB68DB
:102338005A68BB681A43FB685A6006E0FB685B682A
:10234800BA68D2431A40FB685A60BD4604B080BDE3
:1023580080B584B000AF786039600F23FB18002285
:102368001A700023BB603A6880235B04134005D0D1
:102378007B689B680D4A1340BB6002E07B681B6862
:10238800BB60BB683A68134004D00F23FB180122D6
:102398001A7003E00F23FB1800221A700F23FB1892
:1023A8001B78181CBD4604B080BDC046FFFFFFFE69
:1023B80080B582B000AF786039607B683A681A608F
:1023C800BD4602B080BDC04680B584B000AF78601D
:1023D80039600F23FB1800221A700023BB607B684A
:1023E8005B683A681340BB607B681B683A681340B7
:1023F80007D0BB68002B04D00F23FB1801221A70EA
:1024080003E00F23FB1800221A700F23FB181B7818
:10241800181CBD4604B080BD80B582B000AF78609E
:1024280039607B683A681A60BD4602B080BDC04614
:1024380080B500AF80239B02181C0121FEF728FC01
:1024480080235B01181C0121FEF740FC80239B00C0
:10245800181C0121FEF73AFC304B02221A712F4B4F
:1024680000229A712D4BF1221A602C4B03225A71CB
:102478009023DA05294B101C191CFEF7E7FD284BA1
:10248800181CFFF7E1FC264B01221A71244B00228D
:10249800DA60244A224B101C191CFFF7A9FC224BB6
:1024A800181CFEF7C1FF204B00221A801E4B822207
:1024B80052005A801C4BE022D2009A801A4B00220C
:1024C800DA80194B01221A81174B802292005A8117
:1024D800154B08229A81144B0022DA81124B0722ED
:1024E8001A82124A104B101C191CFEF7C1FF0B4B25
:1024F800181CFEF73DFE094B0222DA71074B012238
:102508001A60064B00225A719023DA05034B101CFF
:10251800191CFEF79BFDBD4680BDC0462400002067
:1025280040000020002401402C0000200030014021
:1025380080B500AF62B6FFF77BFF204B181C012166
:10254800FFF712F91E4B1B8801339AB21C4B1A80F5
:102558001C4B1B881C4A934203D11C4B04221A7043
:102568001DE0184B1B881A4A934203D9174B0322C4
:102578001A7014E0134B1B88164A934203D9134B65
:1025880002221A700BE00F4B1B88134A934203D99F
:102598000E4B01221A7002E00C4B00221A70084BF5
:1025A8001B880E4A934207D1084B1B789BB2034AFB
:1025B800101C191CFFF724FAC4E7C046003001407C
:1025C8005A0000205C000020FF0F00005800002087
:1025D8008B0E0000B2090000D9040000983A0000F0
:1025E80030270008000000202400002024000020DC
:1025F80060000020012051E21EFF2F013600003A42
:10260800010050E12200009A020011E12300000AB3
:102618000E0211E38111A0010830A0030130A013BC
:10262800010251E3000051310112A0310332A031FF
:10263800FAFFFF3A020151E3000051318110A03145
:102648008330A031FAFFFF3A0020A0E3010050E1F7
:102658000100402003208221A10050E1A100402078
:10266800A3208221210150E1210140202321822140
:10267800A10150E1A1014020A3218221000050E3E3
:102688002332B0112112A011EFFFFF1A0200A0E1BE
:102698001EFF2FE10100A0030000A0131EFF2FE181
:1026A800010851E32118A0211020A0230020A03305
:1026B800010C51E32114A02108208222100051E3CB
:1026C8002112A02104208222040051E303208282E7
:1026D800A12082903002A0E11EFF2FE1000050E30C
:1026E8000000E013070000EA000051E3FAFFFF0AC8
:1026F80003402DE9BEFFFFEB0640BDE8920003E072
:10270800031041E01EFF2FE11EFF2FE1C046C04627
:10271800C046FDF7D5FCFFF70BFF7047FEE700004A
:082728007847C046B2FFFFEA4A
:10273000006CDC0200000000000000000102030445
:102740000607080900000000010203040102030457
:042750000607080967
:0400000508002715B3
:00000001FF
